:100000009D28AB004230A3000F30A40066200319E6
:100010001210031D1214FC3E031C921003189214BC
:100020004030A3004230A4000F30A700A8011218EE
:1000300037209218372068202303831692008312FA
:100040002308A5002408A6002008A900AA00200F64
:10005000AA018220280895000C309700A71B97164C
:10006000271B17168316061183121215982838209D
:100070000310A70CA40CA30C080083178001840AAA
:10008000FF3E031D3E289828A601A500FF30A507C6
:10009000031CA607031C98280330A400DF3052205D
:1000A0004628A401E83EA300A409FC30031C5B28F9
:1000B000A30703185828A3070000A40F58282318E3
:1000C0006128A31C6528000065280800A801A70175
:1000D0001030A900240DA70DA80D2508A702260899
:1000E000031C260FA80203187C282508A70726084A
:1000F0000318260FA8070310A30DA40DA90B6A2847
:10010000230898281030AC00A401A301AA0CA90C64
:10011000031C90282508A30726080318260FA40708
:10012000A40CA30CA80CA70CAC0B862827089828B5
:100130008313831203130000080007309F0085011A
:10014000203086007C30831685009730860081132E
:1001500020308400603083123E20A0308400503074
:100160003E202030840030303D20C6287F30A00063
:100170000330A600E830A50001300120783044208B
:10018000A001A601A501013001200800A001A601DF
:10019000A50101300120851485130130A6002C3003
:1001A00045200B168B1063000B12851785108618DF
:1001B0002B292F18DC28C6280730B100D030B0001A
:1001C0003108031DE728FA303002031CFD287F3078
:1001D000A0003108A6003008A50001300120061853
:1001E000F228C6280730B00200300318FA28013E72
:1001F0000318FD28B1020318E028A001A601A501FB
:10020000013001200130BA00C9303A020318102928
:100210000530442006180E29B620C628BA0F042936
:10022000B5010130B4003508031D292951303402CD
:100230000318292983160510831205140730A4001A
:10024000D0305220051017304420B40A0319B50FDE
:1002500013292F10C6282F184D292F14B62003302C
:10026000B300E830B200B5010130B4003508031D19
:100270004C295130340203184C298316051083127F
:1002800005143308A400320852200510173044200A
:10029000B40A0319B50F3629C628AF14061DAF10CE
:1002A0000130AF18013EA1000130BA003A08210226
:1002B000031C5F29B62078304420BA0F5629B501B7
:1002C000B40101303502031C6B29031D74292D3044
:1002D0003402031874290A3044200618702974293E
:1002E000B40A0319B50F612901303502031C7F29B7
:1002F000031D7E292D303402031C7F298729030129
:10030000AF1C013E0319AF10031DAF145029AF18E5
:100310008C291430B6008E29C830B6000430330260
:10032000031C9829031DA929753032020318A92935
:1003300083160510831205143308A40032085220D6
:100340000510173044200230B207031C8E29B30F6A
:100350008E290130B70037083602031C662A0130A7
:100360003702031DC629B5010130B4003508031D4D
:10037000C629C93034020318C62932304420061871
:10038000C229D02AB40A0319B50FB62905303302A1
:10039000031CD029031DE429153032020318E42977
:1003A00083160510831205143308A4003208522066
:1003B0000510173044200618DE29D02A0530B20770
:1003C000031CC629B30FC629FF303607A100FF3032
:1003D0000318013EA2002208031D012A210837024A
:1003E000031D012A7F30A0000330A600E830A500DD
:1003F00001300120B4304420A001A601A501013044
:100400000120B5010130B4003508031D142A1A304B
:1004100034020318142A323044200618102AD02A35
:10042000B40A0319B50F042A360837020318402A04
:100430000530B202031CB30304303302031C3F2A0D
:10044000031D262A10303202031C3F2A8316051092
:10045000831205143308A400320852200510173007
:1004600044200618342AD02A0530B202003003187E
:100470003C2A013E03183F2AB30203181C2A642AAF
:100480000230B202031CB30304303302031C642A9B
:10049000031D4E2A10303202031C642A83160510F5
:1004A000831205143308A4003208522005101730B7
:1004B00044200230B20200300318612A013E0318C2
:1004C000642AB3020318442AB70FAB290430B300DF
:1004D0001030B20003303302031C8A2A031D742A31
:1004E000E8303202031C8A2A831605108312051491
:1004F0003308A4003208522005101730442002307F
:10050000B20200300318872A013E03188A2AB30278
:1005100003186A2AB5010130B4003508031DA32A67
:100520000B3034020318A32A831605108312051416
:100530003308A40032085220051017304420B40AB2
:100540000319B50F8D2A85140130BA0004303A0220
:100550000318CF2AA530B9003908A0000930A60039
:10056000C430A500013001203909A1000310210C7D
:10057000AD00AE012E08AA002D08A900A6013C304E
:10058000A5008220A3002808A400230852200130DF
:10059000B9020318AC2AC8304420BA0FA62AC628CC
:1005A000B62003303302031CF12A031DDB2AE83096
:1005B0003202031CF12A8316051083120514330836
:1005C000A400320852200510173044200230B20235
:1005D00000300318EE2A013E0318F12AB302031873
:0405E000D12AC6282E
:02400E00103F61
:00000001FF
